:020000040800F2
:100000000018002069050008E9050008E905000856
:1000100000000000000000000000000000000000E0
:10002000000000000000000000000000E9050008DA
:100030000000000000000000E9050008E9050008D4
:10004000E9050008E9050008E9050008E9050008D8
:10005000E9050008E9050008E9050008E9050008C8
:10006000E9050008E9050008E9050008E9050008B8
:10007000E9050008E9050008E9050008E9050008A8
:10008000E90500080000000000000000E905000884
:1000900000000000E9050008E9050008E90500087E
:1000A00000000000E9050008E9050008E90500086E
:1000B000E905000800000000E9050008E90500085E
:1000C0000448054B10B5834203D0044B002B00D0ED
:1000D000984710BD0004002000040020000000002C
:1000E00006480749091A8910CB0F591810B549104D
:1000F00003D0044B002B00D0984710BD0004002013
:10010000000400200000000010B5074C2378002BED
:1001100009D1FFF7D5FF054B002B02D0044800E0C2
:1001200000BF0123237010BD000400200000000068
:10013000B0230008054B10B5002B03D00449054837
:1001400000E000BFFFF7CCFF10BDC046000000007C
:1001500004040020B023000870B50C4D0C4E761B33
:10016000B61005D0002408CD01349847A642FAD134
:1001700002F01EF9074D084E761BB61005D000247C
:1001800008CD01349847A642FAD170BD002A000874
:10019000002A0008002A0008042A0008F0B505001B
:1001A00083074AD0541E002A44D0CEB20300032253
:1001B00002E00135013C3DD301332E701342F8D1EA
:1001C000032C2FD9FF220A40150215432A04154398
:1001D0000F2C35D92700103F3F093E01B4461E00C1
:1001E0001A0010366644156055609560D56010326F
:1001F000B242F8D10F260C2201373F012640DB190D
:100200003700224217D03E1FB608B400A4461A0099
:100210001C1D644420C2A242FCD103240136B60056
:100220009B193C40002C05D0C9B21C191970013330
:100230009C42FBD1F0BD3400F4E714000300BFE79B
:100240002700E0E7002243088B4274D303098B4266
:100250005FD3030A8B4244D3030B8B4228D3030C96
:100260008B420DD3FF22090212BA030C8B4202D338
:100270001212090265D0030B8B4219D300E0090A60
:10028000C30B8B4201D3CB03C01A5241830B8B4269
:1002900001D38B03C01A5241430B8B4201D34B0352
:1002A000C01A5241030B8B4201D30B03C01A5241B7
:1002B000C30A8B4201D3CB02C01A5241830A8B423C
:1002C00001D38B02C01A5241430A8B4201D34B0225
:1002D000C01A5241030A8B4201D30B02C01A524189
:1002E000CDD2C3098B4201D3CB01C01A524183093D
:1002F0008B4201D38B01C01A524143098B4201D377
:100300004B01C01A524103098B4201D30B01C01AA1
:100310005241C3088B4201D3CB00C01A524183081B
:100320008B4201D38B00C01A524143088B4201D348
:100330004B00C01A5241411A00D2014652411046A8
:100340007047FFE701B5002000F006F802BDC04687
:100350000029F7D076E770477047C046F0B591B0F6
:1003600002AF786036243B193C221A8024257B1981
:10037000324A43CA43C31188198092789A707B68C5
:10038000180000F093FB3A197B681100180000F088
:1003900027FC7B683C21180001F0F6F901F05AFABD
:1003A0007A19012300930F230521002001F0E4FBBB
:1003B0000123019300230093302380221021002089
:1003C00001F0A4FD7B68180001F054FA18203B18D6
:1003D0001B4A12CA12C31188198092789A703A186F
:1003E000012300930B231521032001F0C5FB1020EE
:1003F0003B18144A1168196012791A713A180123CE
:10040000009305232321032001F0B6FB08203B18AD
:100410000D4A1168196012791A713A180123009374
:1004200005232E21032001F0A7FB7B68180001F0B3
:1004300021FAC046BD460FB0F0BDC046C823000833
:10044000D8230008E4230008EC23000890B58BB003
:1004500004AF7860396017243B1900221A70082312
:10046000FB1818000E231A000021FFF797FEFA234D
:100470009B00374A1900100000F054F90023009344
:10048000002302220221132001F06CF800230093C4
:10049000032300220121002001F064F800F0A6F8F7
:1004A000E1235A022B4800230293002301930123E6
:1004B000009313000F22022100F070F9264B254A09
:1004C0001900100000F0B6FA244B224A190010005F
:1004D00000F0B0FA3B1900221A700EE0642000F020
:1004E0003BF9132001F0A0F8642000F035F9172142
:1004F0007B181A787B1801321A701723FB181B78A7
:10050000012BEBD90021132001F0D4F80823FB18AC
:100510001800FFF723FF124B0E4A1900100000F0DD
:1005200089FA104B0B4A1900100000F083FA0C4BAB
:10053000084A1900100000F07DFA642000F00CF960
:10054000132001F071F8642000F006F9F5E7C046C9
:1005500000127A0000440040F4230008FC23000845
:100560001C2400082024000813488546134801680D
:10057000090E134A914205D11248134901601348EC
:100580001349016013481449144A002302E0D45867
:10059000C4500433C4188C42F9D3114A114C0023BF
:1005A00001E013600432A242FBD300F01FF8FFF712
:1005B000D3FDFFF74BFFFEE700180020040000000A
:1005C0001F00000018100240010000000000014060
:1005D000000000000000002000040020082A00089D
:1005E000000400202C040020FEE7000080B500AFCE
:1005F00000F05CF800F082F800F010F872B600F03D
:1006000077F8FA239B00044A1900100000F08AF8DA
:10061000C046BD4680BDC04600127A0080B582B09B
:1006200000AFFB1D01221A701E4B1A681D4B0121E1
:100630000A431A600CE01B4B1B6802221340FA1D90
:10064000F91D09781170022B02D1FB1D00221A70CE
:10065000FB1D1B78002BEED1124B1B68F822934335
:100660001A00104B80210A431A600E4B5A680D4B3A
:10067000F0218A435A600B4B5A680A4B0A490A40D8
:100680005A60084B5A68074B03218A435A60C04698
:10069000044B5B680C221340FAD1C046BD4602B041
:1006A00080BDC04600100240FFF8FFFF80B582B059
:1006B00000AF0E4B9A690D4B01210A439A610B4B17
:1006C0009B69012213407B60084BDA69074B80214C
:1006D00049050A43DA61054BDA6980235B0513405B
:1006E0007B607B68C046BD4602B080BD0010024002
:1006F00080B500AFC046BD4680BD000080B500AFEC
:10070000074B1A68064B01218A431A60C046044B06
:100710001B6801221340FAD1C046BD4680BDC046C9
:100720000020024080B582B000AF7860396039683F
:100730007868FFF787FD03001A00064B013A5A60FC
:10074000044B00229A60034B05221A60C046BD4646
:1007500002B080BD10E000E080B582B000AF0200C2
:10076000BB1D1A800FE00C4B1A6880235B021340FC
:10077000BA1DB91D09881180002B04D0BB1D1A8831
:10078000BB1D013A1A80BB1D1B88002BEBD1C04654
:10079000BD4602B080BDC04610E000E0B0B584B0F8
:1007A00000AFF860080011007B600B243B19021CAD
:1007B0001A700A257B190A1C1A703B191B7818003D
:1007C00000F058F87B191B78180000F069F8FB68F6
:1007D000264A934207D1264BDA69254B80218902AC
:1007E0000A43DA6106E0224B9A69214B8021C90154
:1007F0000A439A61FB6800221A60FB6800225A6073
:10080000FB6800229A607A68FB681100180000F00B
:10081000B1F8182308229446BC4463441A78FB6854
:100820001100180000F052F8202308229446BC441E
:1008300063441A78FB681100180000F0B1F8FB68F7
:100840001A68FB6808210A431A60FB681A68FB688B
:1008500004210A431A60FB681A68FB6801210A43F5
:100860001A60C046BD4604B0B0BDC046004400405A
:100870000010024080B582B000AF0200FB1D1A706C
:10088000FB1D1B780421180000F08CFCFB1D1B785D
:100890000121180000F0B4FDC046BD4602B080BD85
:1008A00080B582B000AF0200FB1D1A70FB1D1B78E3
:1008B0000421180000F076FCFB1D1B7801211800B4
:1008C00000F09EFDC046BD4602B080BD80B582B03E
:1008D00000AF78600A00FB1C1A70FB1C1B78002B11
:1008E0000DD17B681A687B68802149050A431A602C
:1008F0007B681A687B6815490A401A6021E0FB1C76
:100900001B78012B0CD17B681A687B680F490A4061
:100910001A607B681A687B680D490A401A6010E00B
:10092000FB1C1B78022B0CD17B681A687B6808497A
:100930000A401A607B681A687B68802149010A4373
:100940001A60C046BD4602B080BDC046FFEFFFFF43
:10095000FFFFFFEF80B582B000AF78603960396883
:100960007868FFF76FFC03009BB21800BD4602B029
:1009700080BD000080B582B000AF786039603B6810
:10098000064A19001000FFF7E5FF03001A007B6814
:10099000DA60C046BD4602B080BDC04600127A0093
:1009A00080B582B000AF78600A00FB1C1A70FB1C97
:1009B0001B78002B0CD17B689A687B681B490A4026
:1009C0009A607B689A687B6819490A409A6029E0B6
:1009D000FB1C1B78012B07D17B689A687B68802100
:1009E00089000A439A601DE0FB1C1B78022B07D18B
:1009F0007B689A687B68802149000A439A6011E00D
:100A0000FB1C1B78032B0DD17B689A687B688021C7
:100A100089000A439A607B689A687B688021490054
:100A20000A439A60C046BD4602B080BDFFFDFFFF8D
:100A3000FFFEFFFF90B585B000AF786039600E23F0
:100A4000FB1800221A800FE00E243B191B883A681D
:100A5000D3181A787B681100180000F011F83B19C0
:100A60001A883B1901321A800E23FB181B883A683A
:100A7000D3181B78002BE7D1C046BD4605B090BD0A
:100A800080B582B000AF78600A00FB1C1A70C046C7
:100A90007B68DB6980221340FAD07B68FA1C1278ED
:100AA00092B21A85C046BD4602B080BD80B582B004
:100AB00000AF78607B680022DA727B6800221A73CC
:100AC0007B68180000F0EEF87B68180000F066F90B
:100AD0007B680121180000F0FDF97B685A7A7B6879
:100AE0001100180000F0AEF97B681A7A7B681100DB
:100AF000180000F0CDF97B685A787B681100180067
:100B000000F060F97B68DA797B681100180000F06A
:100B100065F97B685A887B681100180000F02CFB8F
:100B20007B689A887B681100180000F030FB7B68B6
:100B3000180000F015F9C046BD4602B080BD90B562
:100B400087B000AFF860B9607A603B60BB6A1A7822
:100B500017217B1801321A70FB6805221A730C00EA
:100B60007B181A78FB681100180000F02FFABA6899
:100B7000FB681100180000F05DFA7A68FB6811004C
:100B8000180000F09FFA3B1900221A700BE03A6837
:100B9000FB681100180000F0AFFA17217B181A78D3
:100BA0007B1801321A70BB6A1B781722BA181278A8
:100BB0009A42ECD3C046FB68180000F0B7FA031E57
:100BC000F9D0FB68180000F0CBF9C046FB681800AC
:100BD00000F0E2F9031EF9D0C046BD4607B090BD53
:100BE00080B582B000AF786039607B6805221A73E7
:100BF0007B680021180000F0E9F93A687B68110071
:100C0000180000F017FA7B68180000F0A1FA031E24
:100C100009D07B680C22DA727B680121180000F091
:100C20000BF8002303E07B680B22DA720123180023
:100C3000BD4602B080BD000080B582B000AF7860D4
:100C40000A00FB1C1A70134B134A19001000FFF71F
:100C5000F1FE124B104A19001000FFF7EBFE0D4B8E
:100C60000D4A19001000FFF7E5FEFB1C1B78012B55
:100C70000BD10B4B084A19001000FFF7DBFE054BA8
:100C8000054A19001000FFF7D5FEC046BD4602B068
:100C900080BDC04638240008004400403C240008C1
:100CA0004824000880B584B002AF78607B681800E3
:100CB00000F034F8184BDA691523190001238B4032
:100CC0001900154B0A43DA617B680222DA720920A7
:100CD00000F036FD0A2000F033FD032300930223C9
:100CE00003220421092000F03DFC0323009302238A
:100CF000032204210A2000F035FC0421092000F021
:100D00007FFB04210A2000F07BFB7B680322DA7260
:100D1000C046BD4602B080BD0010024080B582B022
:100D200000AF78600D4B1A691523190001238B4021
:100D300019000A4B0A431A61084B1A691523190056
:100D400001238B40DB431900044B0A401A617B6886
:100D50000122DA72C046BD4602B080BD00100240DA
:100D600080B582B000AF78600B4B1A680A4B012146
:100D70000A431A607B6802221A73C0467B68180017
:100D800000F00AF9031EF9D07B6803221A73C046EB
:100D9000BD4602B080BDC0460054004080B582B060
:100DA00000AF7860064B1A68054B01218A431A6030
:100DB0007B6800221A73C046BD4602B080BDC046A3
:100DC0000054004080B582B000AF78600A00FB1C80
:100DD0001A70C046BD4602B080BD000080B582B02A
:100DE00000AF78600A00FB1C1A707B685B78002BF0
:100DF0001ED17B68DB79012B0DD10F4B5A680E4B4E
:100E0000802109010A435A600B4B5A680A4B0B496F
:100E10000A405A600CE0084B5A68074B08490A40E0
:100E20005A60054B5A68044B802149010A435A60B5
:100E3000C046BD4602B080BD00540040FFEFFFFF3A
:100E4000FFF7FFFF80B582B000AF78600A00FB1C9F
:100E50001A707B685B7A012B06D10B4B1A680A4B20
:100E60000A490A401A600AE07B685B7A002B06D1C7
:100E7000054B1A68044B802189020A431A60C04658
:100E8000BD4602B080BDC04600540040FFFFFDFFDC
:100E900080B582B000AF78600A00FB1C1A70FB1CA2
:100EA0001B78042B08D89A00074BD3181B689F4661
:100EB000064B074A1A6102E0C04600E0C046C04641
:100EC000BD4602B080BDC04660240008005400400A
:100ED0000E09002080B582B000AF78600A00FB1CCC
:100EE0001A70FB1C1B78002B06D0094B1A68084BA4
:100EF00008490A401A6006E0054B1A68044B802135
:100F000049010A431A60C046BD4602B080BDC046D2
:100F100000540040FFEFFFFF80B582B000AF786063
:100F20000D4B5A680C4B0D490A405A600A4B5A68DF
:100F3000094B802189010A435A60C046064B9A69D1
:100F400080231B021340F9D07B680422DA72C0466A
:100F5000BD4602B080BDC04600540040FFBFFFFF49
:100F600080B582B000AF7860094B5A68084B802189
:100F7000C9010A435A60064B5A68054B05490A40A5
:100F80005A607B680F22DA72C046BD4602B080BD4F
:100F900000540040FFDFFFFF80B582B000AF7860F3
:100FA000094B9A6980231B021A4080231B029A4234
:100FB00004D07B6803221A73012300E00023180089
:100FC000BD4602B080BDC0460054004080B582B02E
:100FD00000AF78600A00FB1C1A70094B5A68084B76
:100FE00008490A405A60064B5A68FB1C1B781B04D0
:100FF0001900034B0A435A60C046BD4602B080BD8B
:1010000000540040FFFF00FF80B582B000AF786061
:10101000064B5A68054B06490A405A607B680A220B
:10102000DA72C046BD4602B080BDC04600540040E2
:10103000FFFBFFFF80B582B000AF78603960134BD3
:101040005A68124B12490A405A607B681800FFF731
:10105000DBFF0E4B59683B681B885B001A00FF23BF
:101060005B001A40094B0A435A607B681800FFF77F
:1010700053FFC0467B68180000F00CF8031EF9D13E
:1010800001231800BD4602B080BDC0460054004098
:10109000FFFFFFFD80B582B000AF7860084B9B6911
:1010A0000122134004D07B680622DA72002303E099
:1010B0007B680522DA7201231800BD4602B080BDAC
:1010C0000054004080B582B000AF786039603B6862
:1010D0001A78084B9A627B680522DA72C0467B68F0
:1010E0001800FFF7D7FF031EF9D1C046BD4602B076
:1010F00080BDC0460054004080B582B000AF78602B
:1011000039603B681A78084B9A627B680522DA726C
:10111000C0467B681800FFF7BDFF031EF9D1C0462B
:10112000BD4602B080BDC0460054004080B582B0CC
:1011300000AF7860054B9B694022134001D001232A
:1011400000E000231800BD4602B080BD00540040FE
:1011500080B582B000AF78600220FFF7FDFA054B42
:101160009B69DBB210221340DBB21800BD4602B00F
:1011700080BDC0460054004080B582B000AF7860AA
:101180000A00BB1C1A80C046BD4602B080BD80B5B7
:1011900082B000AF78600A00BB1C1A80C046BD4612
:1011A00002B080BD80B582B000AF0200FB1D1A7096
:1011B000BB1D0A1C1A70FB1D1B781B09DBB21A0031
:1011C0001C4B9200D3581A68FB1D1B780F210B4053
:1011D0005B00032199400B00DB431800FB1D1B78CB
:1011E0001B09DBB21900134B8900CB5802401A606F
:1011F000FB1D1B781B09DBB21A000E4B9200D35863
:101200001968BB1D1A780C4B9200D258FB1D1B7835
:101210000F2003405B009A40FB1D1B781B09DBB2CB
:101220001800044B8000C3580A431A60C046BD46EC
:1012300002B080BD74240008B024000880B582B0DC
:1012400000AF0200FB1D1A70BB1D0A1C1A70FB1DAB
:101250001B781B09DBB21A001B4B9200D3585A684B
:10126000FB1D1B780F210B40012199400B00DB4334
:101270001800FB1D1B781B09DBB21900124B8900FB
:10128000CB5802405A60FB1D1B781B09DBB21A00C9
:101290000D4B9200D3585968BB1D1A780B4B920026
:1012A000D258FB1D1B780F2003409A40FB1D1B7872
:1012B0001B09DBB21800044B8000C3580A435A6074
:1012C000C046BD4602B080BD74240008F424000866
:1012D00080B582B000AF0200FB1D1A70BB1D0A1C56
:1012E0001A70FB1D1B781B09DBB21A001C4B920005
:1012F000D358DA68FB1D1B780F210B405B000321DC
:1013000099400B00DB431800FB1D1B781B09DBB267
:101310001900134B8900CB580240DA60FB1D1B7883
:101320001B09DBB21A000E4B9200D358D968BB1DC3
:101330001A780C4B9200D258FB1D1B780F200340EB
:101340005B009A40FB1D1B781B09DBB21800044BA5
:101350008000C3580A43DA60C046BD4602B080BD73
:1013600074240008D024000880B582B000AF0200C9
:10137000FB1D1A70BB1D0A1C1A70FB1D1B781B0974
:10138000DBB21A001C4B9200D3589A68FB1D1B78E5
:101390000F210B405B00032199400B001800FB1D3F
:1013A0001B781B09DBB21900134B8900CB58024094
:1013B0009A60FB1D1B781B09DBB21A000E4B9200D2
:1013C000D3589968BB1D1A780C4B9200D258FB1D5C
:1013D0001B780F2003405B009A40FB1D1B781B0904
:1013E000DBB21800044B8000C3580A439A60C04621
:1013F000BD4602B080BDC04674240008E024000849
:1014000080B582B000AF0200FB1D1A703B1D0A1CA4
:101410001A80FB1D1B781B09DBB21800FB1D1B7813
:101420000F2213404D4902018A18D35C19003B1D5D
:101430001B880722D31A19410B000122134002D145
:10144000012000F099F93B1D1B880F2B02D90220C7
:1014500000F092F9FB1D1B78082213403CD1FB1DC4
:101460001B781B09DBB21A003D4B9200D3581A6A55
:10147000FB1D1B780F210B409B000F2199400B0097
:10148000DB431800FB1D1B781B09DBB21900344B32
:101490008900CB5802401A62FB1D1B781B09DBB286
:1014A0001A002F4B9200D3581A6A3B1D1B880F213C
:1014B0001940FB1D1B780F2003409B0099400B0037
:1014C0001800FB1D1B781B09DBB21900244B890097
:1014D000CB5802431A623DE0FB1D1B781B09DBB2AF
:1014E0001A001F4B9200D3585A6AFB1D1B780F211C
:1014F0000B40083B9B000F2199400B00DB43180079
:10150000FB1D1B781B09DBB21900154B8900CB585A
:1015100002405A62FB1D1B781B09DBB21A00104BFC
:101520009200D3585A6A3B1D1B880F211940FB1D9E
:101530001B780F200340083B9B0099400B001800CC
:10154000FB1D1B781B09DBB21900054B8900CB582A
:1015500002435A62BD4602B080BDC04680240008E6
:1015600074240008B0B582B000AF05000C00100074
:101570001900FB1D2A1C1A70BB1D221C1A707B1D32
:10158000021C1A703B1D0A1C1A70FB1D1B781800E8
:1015900000F0D6F8BB1D1A78FB1D1B78110018004F
:1015A000FFF700FE7B1D1A78FB1D1B781100180049
:1015B000FFF744FE3B1D1A78FB1D1B781100180035
:1015C000FFF786FE1823FB181A78FB1D1B78110005
:1015D0001800FFF7C9FEC046BD4602B0B0BD00000E
:1015E00080B582B000AF0200FB1D1A70FB1D1B7896
:1015F0001B09DBB21A000B4B9200D3581B69FA1D72
:1016000012780F210A40012191400A001A40FB1D67
:101610001B780F210B40DA401300DBB21800BD46E7
:1016200002B080BD7424000880B582B000AF020013
:10163000FB1D1A70FB1D1B781800FFF7D1FF031E5E
:101640001AD0FB1D1B781B09DBB21A00184B920045
:10165000D3589969FB1D1B780F2213408022520238
:101660009A40FB1D1B781B09DBB21800104B800051
:10167000C3580A439A6118E0FB1D1B781B09DBB2B3
:101680001A000B4B9200D3589969FB1D1B780F224F
:10169000134001229A40FB1D1B781B09DBB2180086
:1016A000034B8000C3580A439A61BD4602B080BD17
:1016B0007424000880B582B000AF0200FB1D1A70D0
:1016C000BB1D0A1C1A70BB1D1B78002B19D0FB1DFB
:1016D0001B781B09DBB21A00184B9200D35899698A
:1016E000FB1D1B780F22134001229A40FB1D1B7823
:1016F0001B09DBB21800114B8000C3580A439A61E2
:1017000019E0FB1D1B781B09DBB21A000B4B920082
:10171000D3589969FB1D1B780F2213408022520277
:101720009A40FB1D1B781B09DBB21800034B80009D
:10173000C3580A439A61BD4602B080BD74240008B4
:1017400080B582B000AF0200FB1D1A70084B5969CA
:10175000FB1D1B781B09DBB21A00064B9200D25806
:10176000034B0A435A61C046BD4602B080BDC04625
:1017700000100240C424000880B582B000AF02000F
:10178000FB1D1A70FEE7000080B582B000AF7860E4
:101790000A00FB1C1A702E4B1800FFF787F97B68B4
:1017A000180000F03BFC7B680F220021180000F0BD
:1017B0004FFC7B683F21180000F07EFC7B68002115
:1017C000180000F090FC7B680021180000F0A2FCDB
:1017D0007B680221180000F0B6FC7B68002118002D
:1017E00000F0D0FC7B680121180000F0E2FC7B686F
:1017F0000021180000F0F7FC7B681221180000F0AF
:101800000CFD7B689F21180000F01EFD7B68F02115
:10181000180000F030FD7B684021180000F042FD08
:101820007B68A421180000F054FD7B68002118009B
:1018300000F069FD7B680021180000F07EFD7B68E8
:10184000180000F0F8FBC046BD4602B080BDC0469F
:101850001C04002080B500AF8023DA00044B002177
:101860001800FEF79BFC01231800BD4680BDC04652
:101870000000002090B585B002AF254B2121180053
:1018800000F075FD224B0021180000F070FD204B88
:101890007F21180000F06BFD1D4B2221180000F085
:1018A00066FD1B4B0021180000F061FD184B07215D
:1018B000180000F05CFD7B1D01221A70BB1C3C224D
:1018C0001A807B1C40221A70BB1D00221A8014E073
:1018D000BB1D00229A5E0F4BD4187A1CB91C0C4811
:1018E0007B1D00932300FFF72AF9BB1D00229B5E9E
:1018F0009BB201339AB2BB1D1A80BB1D00229B5EB6
:10190000054A9342E4DD01231800BD4603B090BDB3
:101910001C04002000000020FF030000B0B584B0CC
:1019200000AF05000C0010001900BB1D2A1C1A8016
:101930003B1D221C1A80FB1C021C1A70BB1C0A1CBB
:101940001A7009203B1801221A70BB1D1B887F2BBF
:1019500000D983E03B1D1B883F2B00D97EE0BB1DD7
:1019600019883B181A7813005B009B185B00CB1892
:10197000002B00DC72E03B1D1A883B181B78DB0053
:10198000D318002B6ADD0E23FB1800221A805EE0BC
:101990000E23FB1800229B5E052B04D10A23FB18A3
:1019A00000221A8010E0FB1C1A7813009B009B1881
:1019B0001A000E23FB1800215B5ED218294BD318A6
:1019C0001A780A23FB181A800C23FB1800221A80AD
:1019D0002EE00A23FB181B881A000123134017D09E
:1019E0000923FB181B78012B12D10E23FB181A8830
:1019F000BB1D1B88D31898B20C23FB181A883B1DFB
:101A00001B88D31899B2BB1C1B781A0000F02CF865
:101A10000A22BB18BA180021525E52101A800C21FB
:101A20007B1800229B5E9BB201339AB27B181A800E
:101A30000C23FB1800229B5E072BCADD0E217B18AE
:101A400000229B5E9BB201339AB27B181A800E2350
:101A5000FB1800229B5E052B9ADD00E0C046BD46C8
:101A600004B0B0BD0425000890B583B000AF0400F9
:101A700008001100BB1D221C1A803B1D021C1A808D
:101A8000FB1C0A1C1A70BB1D1B887F2B00D96CE045
:101A90003B1D1B883F2B68D8FB1C1B78012B04D0F7
:101AA000022B42D0002B1FD060E0BB1D1A883B1DCB
:101AB0001B88DB0898B20300DB01D3182D4AD35CE6
:101AC0005AB23B1D1B8807210B40012199400B0096
:101AD0005BB2134359B2BB1D1A880300DB01D31854
:101AE000C9B2244AD15441E0BB1D1A883B1D1B8852
:101AF000DB0898B20300DB01D3181E4AD35C5BB24B
:101B00003A1D128807210A40012191400A0052B271
:101B1000D24352B2134059B2BB1D1A880300DB01F5
:101B2000D318C9B2134AD15420E0BB1D1A883B1DFB
:101B30001B88DB0898B20300DB01D3180D4AD35C85
:101B40005AB23B1D1B8807210B40012199400B0015
:101B50005BB2534059B2BB1D1A880300DB01D31896
:101B6000C9B2044AD154C04600E0C046BD4603B0E5
:101B700090BDC04600000020B0B586B000AF0400A4
:101B80000800BA6019000E23FB18221C1A800C23CF
:101B9000FB18021C1A80BB1D0A1C1A8017217B1817
:101BA00000221A707B1800221A7026E00E23FB1800
:101BB0001B88D9B217243B191B781A1C9218D3180A
:101BC000DB18DAB216203B188A181A703B181B78FB
:101BD00098B225003B191B78BA68D3181A782823C5
:101BE000FB181C780C23FB1819882300FFF796FEBE
:101BF0007B191A787B1901321A701723FB181B788E
:101C00009BB2BA1D12889A42D0D8C046BD4606B0D3
:101C1000B0BDB0B584B000AF05000C0010001900D5
:101C2000BB1D2A1C1A803B1D221C1A80BB1C021CD7
:101C30001A803B000A1C1A800E23FB1800221A800F
:101C4000BB1C1B88B42B00D1C0E00CDC2D2B46D074
:101C500002DC002B1ED055E15A2B00D168E0872B07
:101C600000D18AE04EE187225200934200D1FBE08E
:101C700087225200934203DCE12B00D1CBE041E10B
:101C80003C22FF32934200D113E1B422520093422E
:101C900000D037E10E23FB1800221A8016E00E2434
:101CA0003B191A88BB1D1B88D31898B22023FB1838
:101CB0001A783B1D1B881900FFF7D6FE3B1900223E
:101CC0009B5E9BB201339AB23B191A800E23FB181C
:101CD00000229A5E3B001B889A42E0DB12E10E2351
:101CE000FB1800221A801AE00E243B191A88BB1D2B
:101CF0001B88D31898B23B191B883A1D1288D31A37
:101D00009BB22022BA1812781900FFF7ADFE3B19DA
:101D100000229B5E9BB201339AB23B191A800E23BC
:101D2000FB1800229A5E3B001B889A42DCDBE9E04C
:101D30000E23FB1800221A8016E00E243B191B8884
:101D40003A1D1288D31A99B22023FB181A78BB1DAA
:101D50001B881800FFF788FE3B1900229B5E9BB290
:101D600001339AB23B191A800E23FB1800229A5EA7
:101D70003B001B889A42E0DBC4E00E23FB180022E4
:101D80001A801AE00E243B191B88BA1D1288D31A38
:101D900098B23B191B883A1D1288D31A9BB2202295
:101DA000BA1812781900FFF75FFE3B1900229B5EFC
:101DB0009BB201339AB23B191A800E23FB18002202
:101DC0009A5E3B001B889A42DCDB9BE00E23FB18EB
:101DD00000221A8016E00E243B191B88BA1D1288B7
:101DE000D31A98B22023FB181A783B1D1B881900C0
:101DF000FFF73AFE3B1900229B5E9BB201339AB279
:101E00003B191A800E23FB1800229A5E3B001B88A8
:101E10009A42E0DB76E00E23FB1800221A801AE0DB
:101E20000E243B191B88BA1D1288D31A98B23B198D
:101E30001A883B1D1B88D3189BB22022BA1812782F
:101E40001900FFF711FE3B1900229B5E9BB2013384
:101E50009AB23B191A800E23FB1800229A5E3B00AF
:101E60001B889A42DCDB4DE00E23FB1800221A800F
:101E700016E00E243B191A883B1D1B88D31899B213
:101E80002023FB181A78BB1D1B881800FFF7ECFDF8
:101E90003B1900229B5E9BB201339AB23B191A8018
:101EA0000E23FB1800229A5E3B001B889A42E0DB5F
:101EB00028E00E23FB1800221A801AE00E243B199A
:101EC0001A88BB1D1B88D31898B23B191A883B1D72
:101ED0001B88D3189BB22022BA1812781900FFF77A
:101EE000C3FD3B1900229B5E9BB201339AB23B19A2
:101EF0001A800E23FB1800229A5E3B001B889A4230
:101F0000DCDBC046C046BD4604B0B0BDB0B586B04F
:101F100002AF05000C0010001900BB1D2A1C1A801E
:101F20003B1D221C1A80BB1C021C1A803B000A1C91
:101F30001A800E23FB1800221A802023FB181B781E
:101F4000002B43D1BB1C1A883B1D1988BB1D188868
:101F500024257B191B78009313000022FFF759FEFC
:101F60003A1D3B0012881B88D3189BB2013B99B2E3
:101F7000BB1C1A88BB1D18887B191B7800931300A3
:101F80000022FFF746FE3B001C8887235A003B1DBA
:101F90001988BB1D18887B191B7800932300FFF755
:101FA00038FEBA1DBB1C12881B88D3189BB2013B9C
:101FB00098B23B001C8887235A003B1D19887B1967
:101FC0001B7800932300FFF724FE23E00E23FB1869
:101FD00000221A8017E03A1D0E243B1912881B8834
:101FE000D31899B2BB1C1A88BB1D18882423FB1870
:101FF0001B78009313000022FFF70BFE3B191A8891
:102000003B1901321A800E23FA183B0012881B88F4
:102010009A42E0D3C046BD4604B0B0BD80B582B0A0
:1020200000AF78607B68AE21180000F0A0F9C046D0
:10203000BD4602B080BD80B582B000AF78607B68DD
:10204000AF21180000F093F9C046BD4602B080BD34
:1020500080B584B000AF786008001100FB1C021C42
:102060001A70BB1C0A1C1A700F217B1800221A70F0
:10207000BB1C1B780F2B0ED8FB1C1B78102B0AD80F
:10208000BB1C1B781B015AB2FB1C1B785BB21343B1
:102090005AB27B181A707B68D521180000F067F9D6
:1020A0000F23FB181A787B681100180000F05FF905
:1020B000C046BD4604B080BD80B582B000AF786038
:1020C0000A00FB1C1A707B68A821180000F04FF969
:1020D000FB1C1A787B681100180000F048F9C04614
:1020E000BD4602B080BD80B582B000AF78600A0006
:1020F000FB1C1A707B68D321180000F038F9FB1C18
:102100001A787B681100180000F031F9C046BD460E
:1021100002B080BD80B582B000AF78600A00FB1CC1
:102120001A70FB1C1B78072B09D8FB1C1B7840225C
:102130001343DAB27B681100180000F018F9C046AA
:10214000BD4602B080BD80B582B000AF78600A00A5
:10215000FB1C1A707B688D21180000F008F9FB1C2D
:102160001B78012B05D17B681021180000F0FFF8C7
:1021700004E07B681421180000F0F9F8C046BD4661
:1021800002B080BD80B582B000AF78600A00FB1C51
:102190001A707B682021180000F0E9F8FB1C1A78FF
:1021A0007B681100180000F0E2F8C046BD4602B09E
:1021B00080BD80B582B000AF78600A00FB1C1A7049
:1021C000FB1C1B78002B05D07B68A121180000F0B8
:1021D000CEF804E07B68A021180000F0C8F8C046E3
:1021E000BD4602B080BD80B582B000AF78600A0005
:1021F000FB1C1A70FB1C1B78002B05D07B68C021D0
:10220000180000F0B4F804E07B68C821180000F062
:10221000AEF8C046BD4602B080BD80B582B000AF0A
:1022200078600A00FB1C1A707B68DA21180000F045
:102230009EF8FB1C1A787B681100180000F097F8D4
:10224000C046BD4602B080BD80B582B000AF7860A8
:102250000A00FB1C1A707B688121180000F087F8C7
:10226000FB1C1A787B681100180000F080F8C0464B
:10227000BD4602B080BD80B582B000AF78600A0074
:10228000FB1C1A707B68D921180000F070F8FB1C49
:102290001A787B681100180000F069F8C046BD4646
:1022A00002B080BD80B582B000AF78600A00FB1C30
:1022B0001A707B68DB21180000F059F8FB1C1A78B3
:1022C0007B681100180000F052F8C046BD4602B00D
:1022D00080BD80B582B000AF78600A00FB1C1A7028
:1022E000FB1C1B78A42B05D17B68A421180000F0EF
:1022F0003EF804E07B68A521180000F038F8C046DD
:10230000BD4602B080BD80B582B000AF78600A00E3
:10231000FB1C1A70FB1C1B78002B05D07B68A721C7
:10232000180000F024F804E07B68A621180000F0F3
:102330001EF8C046BD4602B080BD80B582B000AF79
:1023400078600A00FB1C1A70FB1C1B78002B05D060
:102350007B682F21180000F00AF804E07B682E212A
:10236000180000F004F8C046BD4602B080BDB0B50C
:1023700086B002AF78600A00FB1C1A700F217B1830
:1023800000221A700E257B1901221A700C203B18AE
:102390003C221A80FC1C7A18391878687B19009343
:1023A0002300FEF7CCFBC046BD4604B0B0BD000024
:1023B000F8B5C046F8BC08BC9E467047F8B5C046A4
:0823C000F8BC08BC9E46704702
:1023C80048656174204D616E6167656D656E740066
:1023D80054656D706572617475726500536574201B
:1023E8003A000000437572203A0000001B5B324A35
:1023F8000000000057656C636F6D6520746F207472
:10240800686520484D4420496E746572666163654D
:102418000A0D00000A0D0000416C6C20497320571A
:102428006F726B696E672066696E65200000000038
:102438000A0D0000493243203A204572726F72003B
:1024480020202D3E20446576696365206E6F7420D8
:10245800466F756E64200000B00E0008BC0E0008C0
:10246800BC0E0008BC0E0008BC0E000800000048A6
:10247800000400480014004870F07070F8F0F6FE90
:10248800F87CF8FCFCE0C0F4F0F010F0F4F0F0F0A8
:10249800F8FCF4E0E0A4A4A0C040000000000000A4
:1024A8000000000000000000030000000000000021
:1024B800010000000300000002000000000002000C
:1024C80000000400000040000000000000000000C0
:1024D80001000000020000000100000000000000F0
:1024E80000000000010000000300000000000000E0
:1024F80001000000000000000100000000000000D2
:10250800003E5B4F5B3E3E6B4F6B3E1C3E7C3E1C71
:10251800183C7E3C181C577D571C1C5E7F5E1C00B7
:10252800183C1800FFE7C3E7FF0018241800FFE76E
:10253800DBE7FF30483A060E2629792926407F0531
:102548000507407F05253F5A3CE73C5A7F3E1C1C47
:1025580008081C1C3E7F14227F22145F5F005F5F07
:1025680006097F017F006689956A606060606094F3
:10257800A2FFA29408047E040810207E20100808F8
:102588002A1C08081C2A08081E101010100C1E0C03
:102598001E0C30383E3830060E3E0E060000000095
:1025A8000000005F00000007000700147F147F147C
:1025B800242A7F2A122313086462364956205000C1
:1025C80008070300001C2241000041221C002A1CAD
:1025D8007F1C2A08083E0808008070300008080898
:1025E8000808000060600020100804023E514945B8
:1025F8003E00427F400072494949462141494D33D6
:102608001814127F1027454545393C4A494931413C
:10261800211109073649494936464949291E00000A
:10262800140000004034000000081422411414145F
:102638001414004122140802015909063E415D594B
:102648004E7C1211127C7F494949363E4141412254
:102658007F4141413E7F494949417F090909013E7E
:10266800414151737F0808087F00417F41002040A5
:10267800413F017F081422417F404040407F021CB7
:10268800027F7F0408107F3E4141413E7F090909CE
:10269800063E4151215E7F0919294626494949329A
:1026A80003017F01033F4040403F1F2040201F3F60
:1026B8004038403F631408146303047804036159E5
:1026C800494D43007F414141020408102000414127
:1026D800417F0402010204404040404000030708D3
:1026E8000020545478407F284444383844444428CF
:1026F800384444287F385454541800087E09021876
:10270800A4A49C787F0804047800447D40002040FD
:10271800403D007F1028440000417F40007C047841
:1027280004787C080404783844444438FC18242489
:102738001818242418FC7C08040408485454542409
:1027480004043F44243C4040207C1C2040201C3C86
:102758004030403C44281028444C9090907C44647D
:10276800544C440008364100000077000000413610
:10277800080002010204023C2623263C1EA1A16196
:10278800123A4040207A38545455592155557941C8
:102798002154547841215554784020545579400C9F
:1027A8001E52721239555555593954545459395580
:1027B8005454580000457C410002457D42000145C3
:1027C8007C40F0292429F0F0282528F07C54554530
:1027D800002054547C547C0A097F493249494932C3
:1027E8003248484832324A4848303A4141217A3AD8
:1027F80042402078009DA0A07D39444444393D40A2
:1028080040403D3C24FF2424487E4943662B2FFC4E
:102818002F2BFF0929F620C0887E090320545479FC
:10282800410000447D413048484A32384040227ACD
:10283800007A0A0A727D0D19317D2629292F28264A
:102848002929292630484D40203808080808080852
:102858000808382F10C8ACBA2F102834FA00007BAB
:10286800000008142A142222142A1408AA00550069
:10287800AAAA55AA55AA000000FF00101010FF00D0
:10288800141414FF001010FF00FF1010F010F014C3
:102898001414FC001414F700FF0000FF00FF1414C8
:1028A800F404FC141417101F10101F101F14141414
:1028B8001F00101010F0000000001F101010101F53
:1028C80010101010F010000000FF10101010101061
:1028D800101010FF10000000FF140000FF00FF00A0
:1028E800001F10170000FC04F41414171017141418
:1028F800F404F40000FF00F714141414141414F76B
:1029080000F7141414171410101F101F141414F4C3
:10291800141010F010F000001F101F0000001F140A
:10292800000000FC140000F010F01010FF10FF145D
:102938001414FF141010101F00000000F010FFFF07
:10294800FFFFFFF0F0F0F0F0FFFFFF0000000000D5
:10295800FFFF0F0F0F0F0F38444438447C2A2A3EDC
:10296800147E02020606027E027E02635549416316
:102978003844443C04407E201E2006027E02029910
:10298800A5E7A5991C2A492A1C4C7201724C304AA9
:102998004D4D303048784830BC625A463D3E494932
:1029A80049007E0101017E2A2A2A2A2A44445F44DA
:1029B8004440514A444040444A51400000FF01030A
:1029C800E080FF000008086B6B08361236243606D4
:1029D8000F090F0600001818000000101000304002
:1029E800FF0101001F01011E00191D1712003C3CC8
:0829F8003C3C0000000000005F
:042A00003501000894
:042A040009010008BC
:102A080000000000000000000000000000000000BE
:102A180000000000000000000000000000000000AE
:102A2800000000000000000000000000000000009E
:102A3800000000000000000000000000000000800E
:102A4800808000000000000000000000000000007E
:102A5800008080C0C00000000000000000000000EE
:102A6800000000000000000000000000000000005E
:102A7800000000000000000000000000000000004E
:102A8800000000000000000000000000000000003E
:102A98000000000080C0E0F0F8FCF8E00000000052
:102AA800000000000000000000000000008080809E
:102AB800808000808000000000808080808000FF8F
:102AC800FFFF000000008080808000008080000000
:102AD80080FFFF8080008080008080808000808070
:102AE8000000000000808000008C8E84000080F8C8
:102AF800F8F880000000000000000000000000005E
:102B0800F0F0F0F0F0F0F0F0F0F0F0F0E0E0C0807D
:102B180000E0FCFEFFFFFF7FFFFFFFFFFF0000005C
:102B28000000000000000000000000FEFFC70101D7
:102B3800010183FFFF00007CFEC70101010183FF43
:102B4800FFFF0038FEC78301010183C7FFFF0000B4
:102B580001FFFF010100FFFF0701010100007FFFE6
:102B680080000000FFFF7F0000FFFFFF000001FF63
:102B7800FFFF01000000000000000000000000004E
:102B8800030F3F7F7FFFFFFFFFFFFFFFE7C7C78FF1
:102B98008F9FBFFFFFC3C0F0FFFFFFFFFFFCFCFCE0
:102BA800FCFCFCFCFCF8F8F0F0E0C00001030303B7
:102BB80003030103030000000001030303030101F1
:102BC80003010000000103030303010103030000E4
:102BD80000030300000003030000000000000001E0
:102BE80003030303030100000001030100000003C5
:102BF80003010000000000000000000000000000C9
:102C080000000080C0E0F0F9FFFFFFFFFF3F1F0F4B
:102C180087C7F7FFFF1F1F3DFCF8F8F8F87C7DFF1A
:102C2800FFFFFFFFFFFFFF7F3F0F0700303000006F
:102C3800000000000000000000000000000000008C
:102C480000000000FEFEFC00000000000000000084
:102C580000000000000000000000000000E0C000CC
:102C680000000000000000000000303000000000FC
:102C7800000000000000000000000000000000004C
:102C880000C0FEFFFFFFFFFFFFFFFFFF7F7F3F1F2B
:102C98000F071F7FFFFFF8F8FFFFFFFFFFFEF8E0B9
:102CA800000000010000000000000000FEFE00001F
:102CB80000FCFEFC0C06060EFCF80000F0F81C0EEA
:102CC8000606060CFFFFFF0000FEFE00000000FCE9
:102CD800FEFC00183C7E66E6CE84000006FFFF0678
:102CE80006FCFEFC0C0606060000FEFE0000C0F80E
:102CF800FC4E4646464E7C7840183C76E6CECC8064
:102D080000000000000000000000000000000000BB
:102D18000000000001070F1F1F3F3F3F3F1F0F0329
:102D28000000000000000000000000000F0F00007D
:102D3800000F0F0F000000000F0F000003070E0C1C
:102D480018180C060F0F0F0000010F0E0C180C0FAF
:102D5800070100040E0C180C0F070000000F0F00ED
:102D6800000F0F0F0000000000000F0F0000000709
:102D7800070C0C181C0C060600040E0C180C0F0788
:102D8800000000000000000000000000000000003B
:102D9800000000000000000000000000000000002B
:102DA800000000000000000000000000000000001B
:102DB800000000000000000000000000000000000B
:102DC80000000000000000000000000000000000FB
:102DD80000000000000000000000000000000000EB
:102DE80000000000000000000000000000000000DB
:102DF80000000000000000000000000000000000CB
:040000050800056981
:00000001FF
